:100000000C94FA000C9417010C9417010C9417012E
:100010000C9417010C9408030C9417010C9417010D
:100020000C9417010C9417010C9417010C941701F0
:100030000C9475170C9417010C9417010C9417016C
:100040000C9417010C94E1020C9417010C94170105
:100050000C9417010C9419010C9417010C941701BE
:100060000C9417010C9417010C9417010C941701B0
:100070000C9417010C9417010C9417010C941701A0
:100080000C9417010C9417010C9417010C94170190
:100090000C941701AA0DAC0DAE0DB00DB20DB40D40
:1000A000B60DB80DBA0DBC0DBE0DC00DC20DC40D00
:1000B000C60DC80DCA0DCC0DCE0DFC0DFC0DFC0DF2
:1000C000FC0DFC0DFC0DD00DD20DD40DD60DD80DB0
:1000D000DA0DDC0DDE0DE00DE20DE40DE60DE80DB0
:1000E000EA0DEC0DEE0DF00DF20DF60D490E4B0E76
:1000F0004D0E4F0E510E530E550E570E590E5B0EF0
:100100005D0E5F0E610E630E650E670E690E6B0E5F
:100110006D0E9B0E9B0E9B0E9B0E9B0E9B0E6F0EF1
:10012000710E730E750E770E790E7B0E7D0E7F0E9F
:10013000810E830E850E870E890E8B0E8D0E8F0E0F
:10014000910E950E090F0F0F150F1B0F210F270F83
:100150002D0F330F390F3F0F450F4B0F510F570F17
:100160005D0F630F690F6F0F750F060F060F060FF8
:10017000060F060F060F7B0F810F870F8D0F930F52
:10018000990F9F0FA50FAB0FB10FB70FBD0FC30F87
:10019000C90FCF0FD50FDB0FE10FE70F37103A1064
:1001A0003D1040104310461049104C104F10521093
:1001B000551058105B105E106110641067106A10C3
:1001C0006D1034103410341034103410341070109A
:1001D0007310761079107C107F10821085108810B3
:1001E0008B108E109110941097109A109D10A010E3
:1001F000A310A61011241FBECFEFD0E1DEBFCDBFEC
:1002000011E0A0E0B1E0E0E3F4E300E00BBF02C0E6
:1002100007900D92A435B107D9F714E0A4E5B1E039
:1002200001C01D92A93BB107E1F70C9423010C9486
:1002300000001F920F920FB60F9211240F900FBE65
:100240000F901F901895CCEFD0E1DEBFCDBF8FEFA0
:1002500084B985B92F980E94650781E897E10E94CB
:10026000B00785E69CE00E94B50781E090E00E941F
:10027000BA07DE011196EBE4F1E083E001900D9204
:100280008150E1F7CE0101960E94AF0B80E091E032
:100290000E944B0C81E191E00E94430C82E491E0CA
:1002A0000E943B0C0E94850B4C0164E670E00E94AA
:1002B000C80760E070E0C4010E94F10A3C0140E020
:1002C00050E0BC01C4010E94E90720EFA22E21E00A
:1002D000B22ECC24DD2490E4E92EF12C02E021E0C2
:1002E00030E041E050E0B301C4010E94860A87E794
:1002F000A82E82E0B82E21E030E041E050E0B301CA
:10030000C4010E94BE0A0E940A071092E1011092E5
:10031000E0011092E3011092E2010E94790C8FEF4C
:1003200087B98AEA88B90E942C0385ED88B90E94B2
:100330002C0380E888B9FFCF0F931F93CF93DF93EF
:10034000EC0181349105B0F08091EC019091ED01C8
:10035000892B81F41092E9011092E801D093EB010E
:10036000C093EA0181E090E09093ED018093EC016D
:10037000C0E4D0E068E08BE20E94500700E010E0AB
:100380000EC0E091E801F091E901E00FF11FEE5C91
:10039000FC4F608189E20E9450070F5F1F4F0C17CE
:1003A0001D0779F78091E0019091E101019749F4EF
:1003B00067E08BE20E9450071092E1011092E00189
:1003C0000AC063E08BE20E94500781E090E09093C6
:1003D000E1018093E001DF91CF911F910F9108958A
:1003E0008091EC019091ED01019771F52091E80168
:1003F0003091E9018091EA019091EB0128173907CA
:1004000018F52091EA013091EB018091E80190917B
:10041000E901281B390B8091E8019091E901805C8A
:100420009F4F9093E9018093E801213431052CF02E
:1004300080E490E00E949C010895C9010E949C0103
:100440001092ED011092EC010895FC011092E90167
:100450001092E8011092ED011092EC0100002F9A29
:100460002081822F82958F7099278230910511F11A
:10047000833091052CF4009761F0019759F516C06F
:1004800084309105F9F084309105C4F0059711F599
:100490001DC0263039F48281813039F5CF010E94A8
:1004A000421723C0CF010E94F30C1FC0CF010E944E
:1004B00084111BC0CF010E94E71217C0CF010E9418
:1004C0002A1413C0CF010E945C150FC0CF010E94F7
:1004D00089180BC02093320383E08093330310927A
:1004E000340383E090E00E949C012F980895CF93FD
:1004F000DF93EC018091E2019091E301019751F5C6
:1005000020E030E0E091E401F091E501E20FF31F1B
:10051000DE01A20FB31F8C91EE50FE4F80832F5F40
:100520003F4F2034310571F78091E4019091E5014E
:10053000805C9F4F9093E5018093E4012091E4015A
:100540003091E5018091E6019091E7012817390784
:10055000A8F11FC01092E5011092E40120E030E004
:10056000E091E401F091E501E20FF31FDE01A20F3B
:10057000B31F8C91EE50FE4F80832F5F3F4F20348E
:10058000310571F73093E5012093E401A981A0348E
:1005900048F41092E3011092E20182EF91E00E9490
:1005A00025020CC081E090E09093E3018093E2018A
:1005B0008A2F99279093E7018093E601DF91CF91ED
:1005C00008951F920F920FB60F9211242F933F930D
:1005D0004F935F936F937F938F939F93AF93BF934B
:1005E000EF93FF930E94C50C80915D0186BDFF9142
:1005F000EF91BF91AF919F918F917F916F915F919B
:100600004F913F912F910F900FBE0F901F90189513
:100610001F920F920FB60F9211242F933F934F9377
:100620005F936F937F938F939F93AF93BF93EF935A
:10063000FF930E94530CFF91EF91BF91AF919F9157
:100640008F917F916F915F914F913F912F910F907B
:100650000FBE0F901F90189520E080E49CE9019751
:10066000F1F72F5F2931C9F70895FF920F931F9378
:10067000162F042FF22E9C01442737FD4095542F4E
:1006800060E472E48FE090E00E94C719215030408E
:10069000163061F0173019F0153019F404C0E1E09C
:1006A00003C0E1E004C0E0E070E002C0E0E071E01F
:1006B000053439F00F3419F451E041E004C050E042
:1006C00001C051E040E082E0F81611F462E001C0A0
:1006D00060E0832F992787FD9A958093C50020932A
:1006E000C40088E18093C100770FEE0FEE0FE72B77
:1006F0005295550F507E5E2B4295407F452B660FDD
:10070000660F660F642B6093C2001F910F91FF90DC
:1007100008951092C50089E18093C40088E1809318
:10072000C10086E08093C20008950895982F8091BB
:10073000C00085FFFCCF9093C60008958091C00053
:1007400087FFFCCF8091C600992708958A3310F463
:10075000805301C087556A3310F4605301C0675558
:100760006F708295807F682B862F99270895FC01F2
:1007700007C08091C00085FFFCCF31969093C600E2
:1007800090819923B1F70895982F92959F70282F03
:100790002F709A3030F48091C00085FFFCCF905DBF
:1007A00005C08091C00085FFFCCF995A9093C60088
:1007B0002A3030F48091C00085FFFCCF205D05C059
:1007C0008091C00085FFFCCF295A2093C600089570
:1007D00087E280939A0485E28093990490E2909353
:1007E0009B0410929C0428E030E030939E042093F8
:1007F0009D0483E28093A60481E28093A5049093F4
:10080000A7041092A8043093AA042093A904089581
:1008100008956091B20481E20E945007089568E053
:100820008BE20E94500761E188E20E94500768E075
:100830008FE20E94500761E18CE20E94500761E064
:100840008FE20E9450071092E1011092E00165E0F2
:1008500083E20E94500708950F931F938C0160E478
:1008600080E20E945007F8016281605884E00E9493
:100870005007F80182818093B1041F910F91089570
:100880000F931F93CF93DF93EC01288539851216C0
:100890001306DCF58E819F81821793071CF568E0B3
:1008A00083E20E94500700E010E00FC08A859B851C
:1008B000E80FF91F608181E20E9450078E819F81BD
:1008C00001969F838E830F5F1F4FEE81FF81888586
:1008D0009985083011051CF4E817F9073CF3E8176F
:1008E000F90724F061E087E20E9450078B81813094
:1008F00031F465E089810E9450071B8206C061E0E7
:1009000089810E94500781E08B83DF91CF911F91F5
:100910000F910895CF93DF93CDB7DEB724970FB62D
:10092000F894DEBF0FBECDBFDC01FC012281338114
:100930001092AC041092AB0481E08093A804832F42
:1009400099278230D9F0833069F1813009F057C09E
:100950008091850499279093AE048093AD0485E837
:1009600094E09093B0048093AF04868197818034A3
:10097000910509F044C088E090E029C0FD0186811E
:1009800097819093AE048093AD04E22FFF27EE0F82
:10099000FF1F8091970490919804E80FF91F8081C0
:1009A000918129C02223C1F0E22FFF27EE0FFF1F04
:1009B0008091F0019091F101E80FF91F0190F08111
:1009C000E02DF093B004E093AF04808199279093D9
:1009D000AE048093AD0413C094E0998383E08A83CE
:1009E00089E08B839C8384E090E09093AE048093B5
:1009F000AD04CE0101969093B0048093AF0485EAD4
:100A000094E00E94400424960FB6F894DEBF0FBE17
:100A1000CDBFDF91CF910895CF93DF9382E20E9403
:100A20002B07C82FDD27C5FF1AC068E083E20E94AC
:100A30005007C6FF10C02091AB043091AC048091E8
:100A4000AD049091AE04281739072CF485EA94E0A0
:100A50000E94400404C061E087E20E945007DF91D9
:100A6000CF9108951F93CF93DF9388E00E942B07C7
:100A7000182FC82FDD27C6FF18C060E085E00E9450
:100A8000500760E884E00E94500760E080E20E9426
:100A9000500768E083E20E94500761E087E20E940D
:100AA000500762E085E00E945007C4FF04C060EC7C
:100AB00089E00E94500717FF04C060ED89E00E94A2
:100AC0005007DF91CF911F9108958AE00E942B0774
:100AD000992780FF03C00E940C05089581FF0DC077
:100AE0008AE20E942B0780917204813061F4E091C8
:100AF0007504F09176040995089582E30E942B070E
:100B00008AE30E942B0708958EE00E942B0768E07D
:100B10008FE20E94500761E08FE20E94500720910F
:100B2000AD043091AE048091A9049091AA0482177B
:100B300093075CF468E083E20E94500761E087E27B
:100B40000E94500781E08093A8040895AF92BF925D
:100B5000CF92DF92EF92FF920F931F93CF93DF9389
:100B6000CDB7DEB728970FB6F894DEBF0FBECDBF66
:100B700086E20E942B0786FF7EC08E010F5F1F4F0B
:100B8000580169E0C62ED12CCC0EDD1E809199044F
:100B90000E942B07F80181938F017501EC15FD056B
:100BA000A9F768E087E20E94500768E083E20E94AC
:100BB000500780E20E942B078F77682F80E20E9407
:100BC000500789819927807690708032910509F4C9
:100BD00040C080349105D1F1892BF1F5F501818177
:100BE0008630D9F0873048F48130F1F18130C8F097
:100BF0008330D1F1853081F521C0893019F18A30F7
:100C000018F4883049F505C08A3071F18B3021F530
:100C100020C0C5010E94090427C0C5010E948A04A2
:100C200023C068E083E20E94500761E081E20E94F5
:100C3000500760E081E20E9450070BC0C5010E948E
:100C40002C0412C0C5010E940F040EC0C5010E94F1
:100C5000080765E083E206C080E20E942B07805807
:100C6000682F80E20E945007F70180818823D1F429
:100C700065E083E215C02091AD043091AE0480910F
:100C8000A9049091AA048217930764F41092AE0409
:100C90001092AD0468E083E20E94500761E087E2B1
:100CA0000E94500728960FB6F894DEBF0FBECDBF46
:100CB000DF91CF911F910F91FF90EF90DF90CF9038
:100CC000BF90AF900895CF92DF92EF92FF920F9373
:100CD0001F93CF93DF93CDB7DEB7C054D0400FB68C
:100CE000F894DEBF0FBECDBF8CE00E942B07992782
:100CF00080FF03C00E94A6057BC081FF2AC08EE250
:100D00000E942B078DE20E942B0789838E010F5FC3
:100D10001F4F6801FFE3EF2EF12CE00EF11E0F5F75
:100D20001F4F0E941907F80180830E151F05B9F7A0
:100D300080915401813031F4E0915701F0915801D4
:100D4000C601099568E08FE20E94500761E08FE2DA
:100D50002BC082FF2CC086E30E942B0785E30E94F4
:100D60002B0789838E010F5F1F4F6801EFE3EE2E83
:100D7000F12CE00EF11E0F5F1F4F0E941907F801C2
:100D800080830E151F05B9F780915501813031F42C
:100D9000E0915901F0915A01C601099568E087E395
:100DA0000E94500761E087E30E94500721C083FF43
:100DB0001FC08EE30E942B078E010F5F1F4F68013B
:100DC00071E4E72EF12CEC0EFD1E8DE30E942B0743
:100DD000F80181938F01EE15FF05B9F78091560157
:100DE000813031F4E0915701F0915801C601099525
:100DF000C05CDF4F0FB6F894DEBF0FBECDBFDF91F2
:100E0000CF911F910F91FF90EF90DF90CF900895B9
:100E10000895089581E080936A0080E18DBB83B3DB
:100E2000876083BB84B3836084BB3F9A479A78947E
:100E3000089588B1805888B984B322E0822784BBA2
:100E40000000000080B198B1905898B994B39227EF
:100E500094BB992708959FEF91B982B988B18058C2
:100E600088B984B395E0892784BB88B1805888B954
:100E700084B3892784BB000011B80E941907992701
:100E8000089582B988B1805888B984B391E08927E0
:100E900084BB88B1805888B984B3892784BB0895FE
:100EA00082B98FEF81B988B1805888B984B395E051
:100EB000892784BB88B1805888B984B3892784BBCB
:100EC000862F0E9441070895089582E1809385044A
:100ED00081E08093860480E191E090938804809380
:100EE00087041092890410928A0410928B0488E07F
:100EF00080938C0410928E0410928D0410929004B2
:100F000010928F0410929204109291041092930404
:100F10001092940410929504109296041092540129
:100F2000109255011092560110927204109273049F
:100F30001092740410927C0410927B041092EF01C2
:100F40001092EE01089590938E0480938D04709317
:100F5000900460938F0450939204409391040895F9
:100F600090938E0480938D040895909390048093C1
:100F70008F04089590939204809391040895809330
:100F80008904089580938A04089580938B040895BA
:100F9000CF93DF939C01CB01E0917B04F0917C0423
:100FA00062E070E00E94B4190FC0A081B18182811B
:100FB000823039F4ED018D8199278217930709F466
:100FC00068870780F085E02D309779F7DF91CF9122
:100FD0000895CF93DF939C01E0917B04F0917C0412
:100FE00014C0A081B1818281843061F48481992709
:100FF0008217930739F4868199278617970711F48A
:10100000ED014B830780F085E02D309751F7DF919C
:10101000CF910895BF92CF92DF92EF92FF920F93FC
:101020001F93CF93DF936C01162FF42EB22EC09135
:101030007B04D0917C042097A1F489E090E00E9489
:10104000BB18FC0190937C0480937B04D182C08206
:10105000138310861782F282B4820583E68215C05C
:10106000EC018F8198850097D9F789E090E00E9484
:10107000BB18FC0198878F83D182C0821383F282D0
:10108000B4820583E68210861782DF91CF911F918B
:101090000F91FF90EF90DF90CF90BF900895EF9267
:1010A000FF921F93CF93DF937C01C091EE01D0910B
:1010B000EF01209711F011E012C085E090E00E944E
:1010C000BB18FC019093EF018093EE01F182E08266
:1010D00012821482138210E012C01F5FEC018B8118
:1010E0009C810097D1F785E090E00E94BB18FC013D
:1010F0009C838B83F182E082128314821382812F7E
:101100009927DF91CF911F91FF90EF900895EF9273
:10111000FF920F931F93CF93DF93E091EE01F09135
:10112000EF0180E090E00380F481E02D019630979C
:10113000D1F7880F991F0E94BB189093F1018093FB
:10114000F0010091EE011091EF01E801E880F980D3
:101150008A81C82FDD27CC0FDD1F8091F00190918F
:10116000F101C80FD91FF701808199270E94BB1890
:101170009983888320E030E017C0E801EA81FF27E7
:10118000EE0FFF1F8091F0019091F101E80FF91F20
:101190000190F081E02DE20FF31FD701A20FB31FE2
:1011A0008C9180832F5F3F4FF7018081992728170B
:1011B00039071CF3E8018B819C81009711F08C01A9
:1011C000C4CFDF91CF911F910F91FF90EF900895C1
:1011D0004F925F926F927F928F929F92AF92BF9247
:1011E000CF92DF92EF92FF920F931F93CF93DF93F3
:1011F000E0917B04F0917C046624772409C082810D
:10120000823019F40894611C711C0780F085E02D70
:101210003097A9F74301880C991CC4010E94BB18A0
:101220009093980480939704E1E0EE2EF12CAA2489
:10123000BB2455C0E0917B04F0917C0479E0C72E7B
:10124000D12C15C0A081B181848199278E159F056D
:1012500019F48381C80ED11CED018D818E1521F406
:101260008281823009F45D010780F085E02D30979E
:1012700049F7009197041091980402501040080D0E
:10128000191DC6010E94BB18F8019183808320E0DC
:1012900030E0E0919704F0919804E80DF91D329741
:1012A0000190F081E02DE20FF31FD501A20FB31FD3
:1012B0008C9180832F5F3F4F2930310551F7E091AA
:1012C0009704F0919804E80DF91D32970190F08190
:1012D000E02D8C2D875F82830894E11CF11C6E1435
:1012E0007F040CF0A7CF61E0C62ED12C59E0A52ECB
:1012F000B12C4424552442E0842E912CA1C0A0910D
:101300007B04B0917C0412C0ED91FC911197818116
:10131000823049F4858199278C159D0521F48481BB
:10132000482E552405C0ED01AF81B885109761F7AF
:1013300031E0E32EF12C79C060917B0470917C0444
:101340006DC0FB01C081D1818981843009F063C007
:10135000868199278E159F0509F05DC084819927A4
:101360008C159D0509F057C0950140E050E0E091D3
:101370009704F0919804E80DF91D32970190F081DF
:10138000E02DE20FF31FDE01A40FB51F8C918083C7
:101390002F5F3F4F4F5F5F4F4930510541F789E065
:1013A00090E0A80EB91EC0917B04D0917C0431C09E
:1013B0008A81853059F58C8199278C159D0531F5E9
:1013C0008D8199278E159F0509F508811981950151
:1013D00040E050E0E0919704F0919804E80DF91D89
:1013E00032970190F081E02DE20FF31FD801A40F96
:1013F000B51F8C9180832F5F3F4F4F5F5F4F47300A
:10140000510541F7E7E0F0E0AE0EBF1E0F80D88532
:10141000C02D209769F6EB016F8178856115710504
:1014200009F08FCF0894E11CF11C4E145F040CF0FE
:1014300083CF0894C11CD11CE2E0F0E08E0E9F1E09
:101440006C147D040CF05BCFDF91CF911F910F9155
:10145000FF90EF90DF90CF90BF90AF909F908F90D4
:101460007F906F905F904F9008956F927F928F92D0
:101470009F92AF92BF92CF92DF92EF92FF920F9323
:10148000CF93DF935C013B014901E0917B04F09134
:101490007C0416C0A081B18184819927A816B90661
:1014A00061F4868199278615970539F48281843005
:1014B00021F4ED018C818F5F8C830780F085E02D16
:1014C000309741F787E090E00E94BB18FC0187E06D
:1014D000808385E0818382820383F582E482C682F1
:1014E000EE24062D2A2D45E067E0CF010E940A0870
:1014F000DF91CF910F91FF90EF90DF90CF90BF9051
:10150000AF909F908F907F906F900895AF92BF9211
:10151000CF92DF92EF92FF920F93FC01A114B104DE
:1015200001F14230510571F04330510599F04130DD
:101530005105B9F481E080937204B0927604A092D0
:1015400075040FC081E080937304B0927804A09278
:10155000770407C081E080937404B0927A04A0926B
:10156000790420583F4FCF010E94350A0F91FF9018
:10157000EF90DF90CF90BF90AF900895AF92BF9261
:10158000CF92DF92EF92FF920F93FC014230510510
:1015900071F04330510599F041305105B9F481E0C3
:1015A00080935401B0925801A09257010FC081E07E
:1015B00080935501B0925A01A092590107C081E071
:1015C00080935601B0925C01A0925B01CF010E9412
:1015D000350A0F91FF90EF90DF90CF90BF90AF90C2
:1015E0000895CF92DF92EF920F931F93CF93DF93E3
:1015F0006C018B01A0917B04B0917C04C0E0D0E031
:1016000014C02D913C911197F90185818C1551F4ED
:10161000FD018281823031F4F90184818F5F8483FE
:10162000C82FDD27FD01A781B085109751F789E00C
:1016300090E00E94BB18FC0189E0808384E08183F4
:101640000283138214821582168217821086EC2E72
:1016500000E02C2D44E069E0CF010E940A08CE0191
:10166000DF91CF911F910F91EF90DF90CF90089570
:10167000BF92CF92DF92EF92FF920F931F93CF937F
:10168000DF936C017B01142FB22EA0917B04B091EB
:101690007C04C0E0D0E014C02D913C911197F90179
:1016A00085818C1551F4FD018281823031F4F9017C
:1016B00084818F5F8483C82FDD27FD01A781B085DA
:1016C000109751F789E090E00E94BB18FC0189E077
:1016D000808384E08183E282138214821583B68240
:1016E00007831086EC2E00E02C2D44E069E0CF014A
:1016F0000E940A08CE01DF91CF911F910F91FF90B8
:10170000EF90DF90CF90BF900895EF920F931F93CB
:10171000109196041F5F1093960489E090E00E9458
:10172000BB18FC0189E0808389E090E09383828389
:1017300082E0818314821583168280EA87838AE19E
:101740008087EE2400E020E042E069E0CF010E94C3
:101750000A08812F99271F910F91EF900895CF9339
:10176000DF93EC01FC0101900020E9F7E81BF90B85
:10177000CF01880F991F0E94BB189C01FE010190A8
:101780000020E9F7EC1BFD0BEE0FFF1FDC01EC93D3
:1017900083E0F901818340E050E009C0FE01E40FDD
:1017A000F51F80818C93FD0111824F5F5F4F129670
:1017B000FE0101900020E9F73197EC1BFD0B4E175D
:1017C0005F0760F3C9010E944F089927DF91CF910D
:1017D0000895EF92FF920F931F93CF93DF938C01A5
:1017E0007B01CA010E94AF0B9C01E0917B04F09148
:1017F0007C0414C0A081B1818281843061F4848131
:1018000099278017910739F4868199278E159F05AE
:1018100011F4ED0128870780F085E02D309751F70E
:10182000DF91CF911F910F91FF90EF9008950F934B
:101830001F93CF93DF938C01CB010E94AF0B9C01D0
:10184000E0917B04F0917C040FC0A081B181828182
:10185000823039F4ED018D8199278017910709F4C1
:101860002E830780F085E02D309779F7DF91CF91B7
:101870001F910F9108950E94AF0B1816190614F4CA
:101880008093950408950E94AF0B1816190614F45E
:101890008093940408950E94AF0B1816190614F44F
:1018A0008093930408951F9386E00E942B07992745
:1018B00086FF03C00E9463060EC082FF03C00E9421
:1018C000650509C081FF03C00E94320504C084FF82
:1018D00002C00E94840587E00E942B07182F60E059
:1018E00087E00E945007612F87E00E9450071F91F8
:1018F00008950E94E8080E9487080E94E80361E0BA
:1019000080E00E94500780E00E942B0780FDFBCF03
:1019100062E081E00E94500760E884E00E94500786
:1019200060E480E20E94500768E083E20E94500772
:1019300069E087E20E9450076FE08DE00E94500747
:101940006FE08BE00E94500768ED89E00E9450072D
:1019500063E38FE00E94500766ED87E00E94500726
:1019600062E085E00E9450076CEC80E00E94500726
:1019700008958EEC80935D0181E080936E008091EC
:101980005D0186BD83E084BD08950895089583E0D8
:101990008093320381E0809333038BE080933403A0
:1019A0002FE62093350393E69093360384E78093E4
:1019B0003703209338039093390381E680933A03E9
:1019C0008EE680933B038FE580933C0380E3809316
:1019D0003D0381E380933E0310923F038EE090E04D
:1019E0000E949C010895FC018081833011F40E94C3
:1019F000C70C0895CF93DF93C1E0D0E08C2F0E94F5
:101A00000B0E2196C431D105C9F7CAE1D0E08C2F65
:101A10000E940B0E2196CD32D105C9F7DF91CF91EF
:101A20000895CF93DF93DC01EC01EA81FB812191E2
:101A30008E81815019F48981E81BF109ED01FB8346
:101A4000EA838E839FB7F8948C9181508C939FBFCB
:101A5000822F9927DF91CF910895FC011082758321
:101A60006483738362834183478346830895CF935E
:101A7000DF93DC019C91ED018981981718F080E0DB
:101A800090E016C0ED01EC81FD8161938F81815062
:101A900019F48981E81BF109ED018F83FD83EC8343
:101AA0009FB7F8948C918F5F8C939FBF81E090E0FB
:101AB000DF91CF910895FC0180818823E9F3CF0164
:101AC0000E94110D99270895FC018081882319F443
:101AD0008FEF9FEF0895CF010E94110D9927089570
:101AE00081E090E0089581E090E0089581E090E049
:101AF000089581E090E00895CF93DF93CDB7DEB7EE
:101B000022970FB6F894DEBF0FBECDBF282F8150AD
:101B1000833120F08951833108F06EC0E22FFF2716
:101B2000EE0FFF1FE35AFE4F82E090E09283818325
:101B3000822F9927AA27BB27FC013197EC32F105A8
:101B400008F05AC0E65BFF4FEE0FFF1F0590F491BF
:101B5000E02D09946D9A47C06E9A49C06F9A43C0B0
:101B6000209A45C0219A3FC0229A41C0239A3BC087
:101B7000249A3DC0259A37C0269A39C0279A33C087
:101B8000509A35C0519A2FC0529A31C0539A2BC0E7
:101B9000549A2DC0559A27C0569A29C0579A23C0E7
:101BA000389A25C0399A1FC03A9A21C03B9A1BC067
:101BB0003C9A1DC03D9A17C03E9A19C0879A13C01F
:101BC000869A15C0859A0FC0849A11C0839A0BC05B
:101BD000829A0DC0819A07C0809A09C0689A03C092
:101BE000699A05C06A9A81E090E008C06B9AE1E0CA
:101BF000F0E0FA83E98304C084E090E09A8389836B
:101C000089819A8122960FB6F894DEBF0FBECDBFB0
:101C1000DF91CF910895982F8150833130F0895111
:101C2000833118F084E090E00895892F0E947C0DA4
:101C300081E090E00895CF93DF93CDB7DEB7229790
:101C40000FB6F894DEBF0FBECDBF282F8150833171
:101C500020F08951833108F06EC0E22FFF27EE0F8C
:101C6000FF1FE35AFE4F81E090E092838183822F31
:101C70009927AA27BB27FC013197EC32F10508F020
:101C80005AC0EA58FF4FEE0FFF1F0590F491E02D68
:101C900009946D9847C06E9849C06F9843C02098CA
:101CA00045C021983FC0229841C023983BC024984A
:101CB0003DC0259837C0269839C0279833C0509822
:101CC00035C051982FC0529831C053982BC05498AA
:101CD0002DC0559827C0569829C0579823C03898CA
:101CE00025C039981FC03A9821C03B981BC03C982A
:101CF0001DC03D9817C03E9819C0879813C086989C
:101D000015C085980FC0849811C083980BC0829825
:101D10000DC0819807C0809809C0689803C0699871
:101D200005C06A9881E090E008C06B98E1E0F0E0BF
:101D3000FA83E98304C084E090E09A8389838981EF
:101D40009A8122960FB6F894DEBF0FBECDBFDF9109
:101D5000CF910895FB011082833091F0843028F4F4
:101D6000813051F0823029F409C0843059F0853037
:101D700059F085E090E0089583B107C086B105C0B1
:101D800089B103C08CB101C08FB1808381E090E044
:101D90000895833091F0843028F4813051F08230FE
:101DA00029F409C0843059F0853069F084E090E06E
:101DB000089565B905C068B903C06BB901C06EB9B3
:101DC00081E090E0089561BB81E090E00895282FC4
:101DD000E82FFF27EE0FFF1FE35AFE4F818192810C
:101DE000029719F086E090E00895822F9927AA279C
:101DF000BB27FC013197EC32F10540F4EE55FF4F63
:101E0000EE0FFF1F0590F491E02D099484E090E01F
:101E10000895662311F0759ADDC07598DBC06623BE
:101E200011F0769AD7C07698D5C0662311F0779ACC
:101E3000D1C07798CFC0662311F0289ACBC02898DC
:101E4000C9C0662311F0299AC5C02998C3C066236A
:101E500011F02A9ABFC02A98BDC0662311F02B9AB0
:101E6000B9C02B98B7C0662311F02C9AB3C02C9838
:101E7000B1C0662311F02D9AADC02D98ABC066237A
:101E800011F02E9AA7C02E98A5C0662311F02F9AA4
:101E9000A1C02F989FC0662311F0589A9BC05898F4
:101EA00099C0662311F0599A95C0599893C066233A
:101EB00011F05A9A8FC05A988DC0662311F05B9A20
:101EC00089C05B9887C0662311F05C9A83C05C98D8
:101ED00081C0662311F05D9A7DC05D987BC066234A
:101EE00011F05E9A77C05E9875C0662311F05F9A14
:101EF00071C05F986FC0662311F0409A6BC0409824
:101F000069C0662311F0419A65C0419863C0662399
:101F100011F0429A5FC042985DC0662311F0439A67
:101F200059C0439857C0662311F0449A53C044984F
:101F300051C0662311F0459A4DC045984BC06623A9
:101F400011F0469A47C0469845C0662311F08F9A13
:101F500041C08F983FC0662311F08E9A3BC08E9887
:101F600039C0662311F08D9A35C08D9833C0662331
:101F700011F08C9A2FC08C982DC0662311F08B9A8B
:101F800029C08B9827C0662311F08A9A23C08A98AB
:101F900021C0662311F0899A1DC089981BC0662351
:101FA00011F0889A17C0889815C0662311F0709AAE
:101FB00011C070980FC0662311F0719A0BC0719810
:101FC00009C0662311F0729A05C0729803C0662397
:101FD00021F0739A81E090E00895739881E090E099
:101FE00008951F93182F8150833130F08951833128
:101FF00018F084E090E013C0E12FFF27EE0FFF1FE1
:10200000E35AFE4F83E090E092838183812F0E9408
:102010007C0D61E0812F0E94E70E81E090E01F912E
:102020000895CF93DF93282FEB011882E82FFF2725
:10203000EE0FFF1FE35AFE4F81819281019719F045
:1020400086E090E089C0822F9927AA27BB27FC0150
:102050003197EC32F10540F4E253FF4FEE0FFF1FD2
:102060000590F491E02D099484E090E075C0659BA3
:1020700071C06EC0669B6EC06BC0679B6BC068C052
:10208000189B68C065C0199B65C062C01A9B62C07E
:102090005FC01B9B5FC05CC01C9B5CC059C01D9B8C
:1020A00059C056C01E9B56C053C01F9B53C050C042
:1020B000489B50C04DC0499B4DC04AC04A9B4AC036
:1020C00047C04B9B47C044C04C9B44C041C04D9B44
:1020D00041C03EC04E9B3EC03BC04F9B3BC038C042
:1020E000309B38C035C0319B35C032C0329B32C0C6
:1020F0002FC0339B2FC02CC0349B2CC029C0359BD4
:1021000029C026C0369B26C023C07F9B23C020C089
:102110007E9B20C01DC07D9B1DC01AC07C9B1AC029
:1021200017C07B9B17C014C07A9B14C011C0799B49
:1021300011C00EC0789B0EC00BC0609B0BC008C0C6
:10214000619B08C005C0629B05C002C0639B02C0C2
:1021500081E0888381E090E0DF91CF910895CF9373
:10216000DF93CDB7DEB721970FB6F894DEBF0FBE71
:10217000CDBF9BE190933203BE016F5F7F4F0E9402
:1021800011108093330389818093340383E090E0BE
:102190000E949C0121960FB6F894DEBF0FBECDBF02
:1021A000DF91CF9108959AE1909332030E94E70E58
:1021B000809333031092340383E090E00E949C01EB
:1021C000089598E1909332030E94C90E80933303DF
:1021D0001092340383E090E00E949C010895982FB0
:1021E00089E180933203933099F0943028F4913050
:1021F00059F0923029F40AC0943061F0953061F0C2
:1022000085E090E020E00BC023B107C026B105C0F7
:1022100029B103C02CB101C02FB181E090E08093BF
:1022200033032093340383E090E00E949C010895DF
:1022300097E1909332030E94F10F80933303109241
:10224000340383E090E00E949C01089595E190930F
:1022500032030E941B0E809333031092340383E0F9
:1022600090E00E949C01089596E1909332030E94B1
:102270007C0D809333031092340383E090E00E943E
:102280009C01089584E18093320381E080933303BD
:102290001092340383E090E00E949C01089582E153
:1022A0008093320381E0809333031092340383E000
:1022B00090E00E949C01089583E18093320381E0C5
:1022C000809333031092340383E090E00E949C01DA
:1022D000089580E18093320381E08093330310926C
:1022E000340383E090E00E949C01089591E1909373
:1022F00032030E940B0E809333031092340383E069
:1023000090E00E949C010895FC0180818531C9F113
:10231000863180F4823131F1833130F48031D1F073
:10232000813109F04CC01AC0833109F1843109F0C0
:1023300046C022C0883189F1893128F4863129F1DB
:102340008731E9F526C08A3189F18A3158F18B311C
:10235000B1F531C082810E946911089582810E9485
:1023600076110895638182810E944F1108956381DF
:1023700082810E945C110895638182810E944211D2
:10238000089582810E942611089582810E9434114D
:10239000089582810E9418110895638182810E94AC
:1023A000E110089582810E94EF1008956381828177
:1023B0000E94D310089582810E94AF1008958093E7
:1023C000320383E0809333031092340383E090E080
:1023D0000E949C010895FC018197089718F084E001
:1023E00090E00895EE0FFF1FE35AFE4F84E090E067
:1023F0009283818381E090E0089510927C00823086
:10240000910541F08330910569F0019741F082E038
:1024100090E0089580917C00806480937C0081E04E
:1024200090E0089580917C00806C80937C0081E036
:1024300090E0089593E890937A0090917C00907FCB
:10244000982B90937C0080917A00806480937A002E
:1024500080917A0086FDFCCF809178009091790080
:1024600020E030E040E050E080917A00806480938A
:102470007A0080917A0086FDFCCF8091780090915F
:102480007900480F591F2F5F3F4F2430310561F706
:1024900080917A008F7780937A00CA01969587950C
:1024A000969587950895CF93DF939C01EB01198250
:1024B0001882FC01EE0FFF1FE35AFE4F81819281CB
:1024C000049719F086E090E03CC02432310541F1D8
:1024D0002532310554F42232310541F123323105E0
:1024E00014F52132310569F424C02632310591F00A
:1024F0002632310594F02732310549F02832310572
:1025000019F087E090E01DC080E090E014C081E009
:1025100090E011C082E090E00EC083E090E00BC03C
:1025200084E090E008C085E090E005C086E090E09F
:1025300002C087E090E00E941A129983888381E0AC
:1025400090E0DF91CF91089522E2209332030E9420
:10255000FD118093330382E090E00E949C01089576
:10256000CF93DF93CDB7DEB722970FB6F894DEBFD7
:102570000FBECDBF21E220933203BE016F5F7F4FBC
:102580000E9453128093330329813A81832F992724
:10259000809334032093350384E090E00E949C01F3
:1025A00022960FB6F894DEBF0FBECDBFDF91CF915C
:1025B000089520E2209332030E94EB1180933303AD
:1025C0001092340383E090E00E949C010895FC0186
:1025D0008081813249F0823261F0803279F48281E7
:1025E00099270E94D9120895828199270E94B012DA
:1025F0000895828199270E94A4120895809332033E
:1026000083E0809333031092340383E090E00E94D0
:102610009C0108958091B9009927887F9070089552
:102620008091BC0087FFFCCF0895ECEBF0E0808147
:10263000846080838BE090E09093770180937601B3
:102640008CE090E0909379018093780181E090E0B4
:102650000895ECEBF0E080818B7F808382E090E056
:10266000909377018093760190937901809378011C
:1026700081E090E008958130910511F48CE00BC069
:102680008230910511F488E106C0039719F082E0C9
:1026900090E0089588E48093B8008091B9008C7F21
:1026A0008093B9008091B9008093B90081E090E0F7
:1026B00008958091B90084EA8093BC008091BC00A9
:1026C00087FFFCCF81E090E0089584E98093BC000F
:1026D00081E090E008958093BB0084E88093BC0083
:1026E0008091BC0087FFFCCF80E090E0089584E8F3
:1026F0008093BC008091BC0087FFFCCF8091BB0021
:102700009927089585E38093320381E08093330312
:102710008093340384E88093BC008091BC0087FFE1
:10272000FCCF8091BB008093350385E090E00E9450
:102730009C01089540E050E00FC0F901E40FF51F3F
:1027400080818093BB0084E88093BC008091BC00B2
:1027500087FFFCCF4F5F5F4F4617570774F384E343
:102760008093320381E0809333031092340383E03B
:1027700090E00E949C01089587E38093320384E9EE
:102780008093BC0081E0809333031092340383E094
:1027900090E00E949C01089586E38093320380912B
:1027A000B90084EA8093BC008091BC0087FFFCCF15
:1027B00081E0809333031092340383E090E00E9421
:1027C0009C01089522E3209332030E943B138093DF
:1027D00033031092340383E090E00E949C0108953B
:1027E00081E380933203ECEBF0E080818B7F808388
:1027F00082E090E090937701809376019093790145
:102800008093780181E0809333031092340383E056
:1028100090E00E949C01089580E380933203ECEBEA
:10282000F0E08081846080838BE090E0909377017A
:10283000809376018CE090E0909379018093780109
:1028400081E0809333031092340383E090E00E9490
:102850009C010895FC0180818433D9F0853338F4DC
:10286000813379F0823381F0803389F507C0863374
:1028700041F18633D8F0873351F526C00E940C14FD
:1028800008950E94F0130895828199270E94E2130F
:102890000895428155276181772764507040838174
:1028A00034969F0199270E949A13089542815527D3
:1028B0006181772764507040838199270E94821339
:1028C00008950E94CC1308950E94BC13089580932C
:1028D000320383E0809333031092340383E090E06B
:1028E0000E949C01089585B1817F85B9239886E077
:1028F00084B91CBC1DBC83E58CBD88E090E090933E
:102900006901809368018AE090E090936B01809365
:102910006A0189E090E090936D0180936C0181E001
:1029200090E008951CBC1DBC82E090E0909369018A
:102930008093680190936B0180936A0190936D017D
:1029400080936C0181E090E00895089581E090E02B
:102950000895AC0120E030E00AC0FA01E20FF31F55
:1029600080818EBD0DB407FEFDCF2F5F3F4F261730
:1029700037079CF381E090E00895DC0120E030E02F
:1029800040E050E015C01EBC09C04F5F5F4F83E0C0
:10299000493E58071CF088E090E008950DB407FE0A
:1029A000F4CFFD01E20FF31F8EB580832F5F3F4F01
:1029B0002617370744F381E090E00895CF93DF9323
:1029C000EC0120E030E0A0E0B0E018C0FE01E20F32
:1029D000F31F80818EBD08C0119683E0A93EB80721
:1029E0001CF088E090E00FC00DB407FEF5CFFB01AE
:1029F000E20FF31F8EB580832F5F3F4F24173507FB
:102A00002CF381E090E0DF91CF9108950F931F9315
:102A10008B0123E420933203AB0164E373E00E9453
:102A2000DE148093330310923403C80102960E948F
:102A30009C011F910F9108950F931F938C0184E4C3
:102A400080933203B80184E393E00E94BD14809325
:102A5000330310923403C80102960E949C011F9117
:102A60000F91089523E4209332030E94A9148093C8
:102A700033031092340383E090E00E949C01089598
:102A800081E4809332030E94921480933303109266
:102A9000340383E090E00E949C01089580E48093D9
:102AA00032030E947314809333031092350383E042
:102AB00090E00E949C010895CF93DF93EC01888100
:102AC0008334A1F0843438F4813469F0823458F5C9
:102AD0008034F1F405C0843481F08534C9F411C028
:102AE0000E944E1520C00E9440151DC069817727A5
:102AF000CE0102960E94321516C0898199270E9444
:102B00001C1569817727CE0102960E9406150BC01D
:102B10008093320383E0809333031092340383E085
:102B200090E00E949C01DF91CF910895209A219A14
:102B3000229A2398249A259A2C982D9882E090E046
:102B40009093850180938401909383018093820107
:102B5000909381018093800181E090E090937F01C8
:102B600080937E01089582E090E0909369018093C4
:102B7000680190936B0180936A0190936D0180933B
:102B80006C0181E090E00895289829982A9880E2C5
:102B90009EE40197F1F7289A8AE0982F9A95F1F729
:102BA0002A9A299A8A95F1F70895282F299887FD5E
:102BB00002C02A9801C02A9A8AE0982F9A95F1F7C4
:102BC000299A8A95F1F7299826FF02C02A9A01C00E
:102BD0002A988AE0982F9A95F1F7299A8A95F1F721
:102BE0000895282F220F30E0299827FF02C02A9A43
:102BF00001C02A988AE0982F9A95F1F7299A8A9528
:102C0000F1F73F5F373011F0220FEECF0895282FF4
:102C100030E0299827FF02C02A9A01C02A988AE04A
:102C2000982F9A95F1F7299A8A95F1F73F5F3830F6
:102C300011F0220FEECF089529982A988AE0982F54
:102C40009A95F1F7299A982F9A95F1F7299828984B
:102C5000982F9A95F1F7299A982F9A95F1F7299834
:102C60008A95F1F7289A80E090E0089529982898AD
:102C70002A982B9A08950E94C41580E30E94D515C6
:102C800080E60E94F11508950E94C41580E00E941C
:102C9000D51580E00E94F1150E94361608950F9315
:102CA0001F93182F062F0E94C41580E40E94D5158B
:102CB000812F0E94F115802F0E94071681E090E07D
:102CC0001F910F9108951F93182F0E94C41580EC37
:102CD0000E94D515812F0E94F1150E941C1699277C
:102CE0001F91089529988AE08A95F1F72A9830E093
:102CF00090E0990F299A2AE0822F8A95F1F7299876
:102D00001B999F5F822F8A95F1F73F5F383089F7D3
:102D10002898299A822F8A95F1F7289A29982A9536
:102D2000F1F7892F992708951F93182F0E94C41532
:102D300080E80E94D515812F0E94F1150E9472161D
:102D400099271F910895DF92EF92FF920F931F939F
:102D5000CF93DF93D82E7B018A01C0E0D0E009C079
:102D60008D2D8C0F0E949416F801EC0FFD1F8083AF
:102D70002196CE15DF05A1F781E090E0DF91CF919C
:102D80001F910F91FF90EF90DF9008950F931F9385
:102D9000082F162F0E943B16612F802F0E944F167E
:102DA00081E090E01F910F910895DF92EF92FF92E2
:102DB0000F931F93CF93DF93D82E7B018A01C0E03E
:102DC000D0E009C0F801EC0FFD1F60818D2D8C0F44
:102DD0000E94C6162196CE15DF05A1F781E090E08E
:102DE000DF91CF911F910F91FF90EF90DF900895A9
:102DF00094E0909332030E94D5168093330310928F
:102E0000340383E090E00E949C0108950F931F9388
:102E10008B0193E09093320344E353E00E94A316A6
:102E200080933303C80102960E949C011F910F9169
:102E3000089582E08093320382E090E090936901EC
:102E40008093680190936B0180936A0190936D0168
:102E500080936C0181E0809333031092340383E00C
:102E600090E00E949C01089581E0809332030E94CB
:102E70009615809333031092340383E090E00E9410
:102E80009C010895FC018381823069F0833018F43D
:102E90008130F1F405C0833049F08430C9F40FC0AB
:102EA0000E94341708950E9419170895AF014A5FD0
:102EB0005F4F6581772784810E9406170895AF01CF
:102EC0004A5F5F4F6581772784810E94F8160895D5
:102ED00080818093320383E0809333031092340324
:102EE00083E090E00E949C0108951F920F920FB61C
:102EF0000F9211240F900FBE0F901F9018959C01F8
:102F00000897029718F084E090E00895F901EE0F19
:102F1000FF1FE35AFE4F8DE090E0928381832830BB
:102F2000310531F02930310531F087E090E0089526
:102F300081E090E00895259A81E090E090938900E7
:102F40008093880081E88093800089E080938100ED
:102F500081E090E008959C01FC01EE0FFF1FE35A11
:102F6000FE4F818192810D9719F086E090E00895DF
:102F70002830310539F12930310519F087E090E02A
:102F8000089563307105B1F06430710544F4613027
:102F9000710561F06230710509F040C009C064300C
:102FA000710551F065307105C9F508C081E007C0B1
:102FB00082E005C083E003C084E001C085E0809327
:102FC000810029C064307105E9F06530710554F461
:102FD0006230710599F06330710594F461307105C8
:102FE000E9F40AC06630710589F06630710564F055
:102FF0006730710599F40CC089E60BC08AE609C0F8
:103000008BE607C08CE605C08DE603C08EE601C0E6
:103010008FE68093B00081E090E0089581E090E039
:1030200008959C01FC01EE0FFF1FE35AFE4F8181C2
:1030300092810D9719F086E090E0089528303105CF
:1030400069F02930310519F087E090E00895709318
:1030500089006093880081E090E008956093B30058
:1030600081E090E0089523E5209332030E94111837
:10307000809333031092340383E090E00E949C011C
:10308000089522E5209332030E94AB178093330307
:103090001092340383E090E00E949C01089520E5A3
:1030A000209332030E947F178093330310923403DE
:1030B00083E090E00E949C0108959C01FC01EE0FCA
:1030C000FF1FE35AFE4F82E090E092838183283015
:1030D000310531F02930310531F086E090E0089576
:1030E0001092B00002C010928100822F0E947C0DCD
:1030F00081E090E0089521E5209332030E945D185D
:10310000809333031092340383E090E00E949C018B
:103110000895FC018081813579F0823518F480357D
:10312000F1F405C0823569F08335C9F411C082819C
:1031300099270E944F180895828199270E947B1831
:10314000089563817727828199270E944118089505
:1031500063817727828199270E943318089580938D
:10316000320383E0809333031092340383E090E0D2
:103170000E949C010895CF93DF93AC01029710F455
:1031800042E050E0A091B704B091B804FD01C0E066
:10319000D0E020E030E020C0808191818417950745
:1031A00069F482819381209719F09B838A8304C0FC
:1031B0009093B8048093B704CF0132C048175907E1
:1031C00038F42115310519F08217930708F49C0192
:1031D000EF010280F381E02D3097F1F621153105E2
:1031E00089F1C901841B950B049708F4A901E0E05B
:1031F000F0E026C08D919C91119782179307E9F416
:103200004817590779F4ED018A819B81309719F0AD
:103210009383828304C09093B8048093B704CD0154
:10322000029649C0841B950BFD01E80FF91F4193DD
:10323000519302978D939C933AC0FD01A281B38173
:103240001097C1F68091B5049091B604892B41F492
:1032500080915001909151019093B6048093B504F0
:1032600020915201309153012115310541F42DB7C0
:103270003EB780914E0190914F01281B390BE09190
:10328000B504F091B6042E1B3F0B2417350788F0C8
:10329000CA0102962817390760F0CF01840F951FE5
:1032A00002969093B6048093B50441935193CF0155
:1032B00002C080E090E0DF91CF910895CF93DF933B
:1032C000009709F44EC0EC0122971B821A82A0914C
:1032D000B704B091B804109711F140E050E001C07C
:1032E000DC01AC17BD0700F1BB83AA83FE0121916D
:1032F0003191E20FF31FEA17FB0771F42E5F3F4F86
:103300008D919C911197820F931F99838883FD0162
:10331000828193819B838A834115510559F4D0930F
:10332000B804C093B7041DC0FD0182819381AD0133
:103330000097B1F6FA01D383C28321913191E20F54
:10334000F31FEC17FD0769F42E5F3F4F88819981C9
:10335000820F931FFA01918380838A819B819383DB
:103360008283DF91CF91089597FB092E07260AD01B
:1033700077FD04D027D006D000201AF4709561950F
:103380007F4F0895F6F7909581959F4F089597FB8D
:10339000092E05260ED057FD04D028D00AD0001CD7
:1033A00038F450954095309521953F4F4F4F5F4FE2
:1033B0000895F6F790958095709561957F4F8F4FA2
:1033C0009F4F0895AA1BBB1B51E107C0AA1FBB1F3B
:1033D000A617B70710F0A61BB70B881F991F5A95A1
:1033E000A9F780959095BC01CD010895A1E21A2E10
:1033F000AA1BBB1BFD010DC0AA1FBB1FEE1FFF1F99
:10340000A217B307E407F50720F0A21BB30BE40BE8
:10341000F50B661F771F881F991F1A9469F760952F
:103420007095809590959B01AC01BD01CF010895E9
:10343000456D62656464656450726F6A6563747338
:10344000004F63746F70757355534220496E7465F5
:10345000726661636520436F6E7665727465722073
:10346000616E6420492F4F20457874656E73696FD3
:103470006E0032303038313130380009040020001D
:04348000B90400008B
:00000001FF
